:020000040000FA
:02000000A02836
:08000800A000030EA100831209
:1000100006181028831601178312B23081002D288C
:1000200083160113831203140B190310A20DA30DE1
:10003000A40DA50DA60DA70DB70B2D283030B700C8
:100040002E152708AD002608AC002508AB002408B3
:10005000AA002308A9002208A8008B100B11210E6A
:080060008300A00E200E090030
:10014000203084008001840A80300402031CA2282D
:100150003830840060218000B30A840A78300402B9
:10016000031CAA284030B1003830B0007830AF000E
:100170008316FE308505333086058312850186019E
:1001800007309F00C8308316810083123130900001
:100190007E309200A630831698008312803098003B
:1001A0000C30831699008312003083168C00831262
:1001B00090308B0081018E018F010B118B100B1081
:1001C0008C130C138C120C120C118C100C108B173E
:1001D0000F212E191C218E1FE8288F018E018E16EB
:1001E0000E1647210510B60BE8280A30B60011217B
:1001F000063031020318E828AA30B2003721AA30AD
:10020000B2003721AA30B20037216430B200372162
:100210003508B20037216530B2003721E828640084
:1002200008000039851C0838051E0438851D023871
:10023000051D0138B50008002E110608803A860019
:1002400005148E018F010C102D08B20037212C08E7
:10025000B20037212B08B20037212A08B20037211B
:100260002908B20037212808B20037210800483099
:10027000310203180617031808002F0884003208FB
:100280008000B10AAF0A3830AF1BAF0008000C1E67
:100290000800B1080319080030088400000899001C
:1002A000B103B00A3830B01BB0000800B3130430FB
:1002B0008A0033088200B31704308A0033088200B2
:0C02C000B317331307308A0033088200A4
:1008000030343034303430343034303430343034C8
:1008100030343034313431343134313431343134B2
:10082000313431343134313432343234323432349C
:100830003234323432343234323432343334333486
:100840003334333433343334333433343334333470
:100850003434343434343434343434343434343458
:100860003434343435343534353435343534353442
:10087000353435343534353436343634363436342C
:100880003634363436343634363436343734373416
:100890003734373437343734373437343734373400
:1008A00038343834383438343834383438343834E8
:1008B00038343834393439343934393439343934D2
:1008C00039343934393439343034303430343034E4
:1008D00030343034303430343034303431343134F6
:1008E00031343134313431343134313431343134E0
:1008F00032343234323432343234323432343234C8
:1009000030343134323433343434353436343734AB
:100910003834393430343134323433343434353497
:100920003634373438343934303431343234333483
:10093000343435343634373438343934303431346F
:10094000323433343434353436343734383439345B
:10095000303431343234333434343534363437345B
:100960003834393430343134323433343434353447
:100970003634373438343934303431343234333433
:10098000343435343634373438343934303431341F
:10099000323433343434353436343734383439340B
:1009A000303431343234333434343534363437340B
:1009B00038343934303431343234333434343534F7
:1009C00036343734383439343034313432343334E3
:1009D00034343534363437343834393430343134CF
:1009E00032343334343435343634373438343934BB
:1009F00030343134323433343434353436343734BB
:100A00003D34003405340134003400340034003403
:100A1000D5340034DD34D9346934003471346D3464
:100A20000034003400340034003400340034003426
:100A30000034003400340034003400340034003416
:100A4000453400344D34493400340034003400342B
:100A50001D34003425342134B1340034B934B53474
:100A60002134003429342534003400340034003477
:100A7000F93400340134FD348D340034953491342C
:100A800000340034003400340034003400340034C6
:100A900000340034003400340034003400340034B6
:100AA00000340034003400340034003400340034A6
:100AB0000034003400340034003400340034003496
:100AC0000034003400340034003400340034003486
:100AD0000034003400340034003400340034003476
:100AE0000034003400340034003400340034003466
:100AF0000034003400340034003400340034003456
:100B0000153400341D3419340034003400340034FA
:100B1000ED340034F534F1348134003489348534D3
:100B20000034003400340034003400340034003425
:100B30000034003400340034003400340034003415
:100B40005D340034653461340034003400340034E2
:100B5000353400343D343934C9340034D134CD34E3
:100B60003934003441343D3400340034003400342E
:100B70001134003419341534A5340034AD34A9349B
:100B80000934003411340D3400340034003400349E
:100B9000E1340034E934E534753400347D3479349B
:100BA00000340034003400340034003400340034A5
:100BB0000034003400340034003400340034003495
:100BC0005134003459345534003400340034003486
:100BD0002934003431342D34BD340034C534C134AB
:100BE0002D340034353431340034003400340034D2
:100BF000053400340D34093499340034A1349D3463
:100C00000134FF3400340034FF34FF34FF34FF3448
:100C10000034FF34003400340034FF340034003436
:100C2000FF34FF34FF34FF34FF34FF34FF34FF342C
:100C3000FF34FF34FF34FF34FF34FF34FF34FF341C
:100C40000034FF3400340034FF34FF34FF34FF3409
:100C50000134FF34013401340034FF3400340034F3
:100C60000034FF3400340034FF34FF34FF34FF34E9
:100C70000034FF34013400340034FF3400340034D5
:100C8000FF34FF34FF34FF34FF34FF34FF34FF34CC
:100C9000FF34FF34FF34FF34FF34FF34FF34FF34BC
:100CA000FF34FF34FF34FF34FF34FF34FF34FF34AC
:100CB000FF34FF34FF34FF34FF34FF34FF34FF349C
:100CC000FF34FF34FF34FF34FF34FF34FF34FF348C
:100CD000FF34FF34FF34FF34FF34FF34FF34FF347C
:100CE000FF34FF34FF34FF34FF34FF34FF34FF346C
:100CF000FF34FF34FF34FF34FF34FF34FF34FF345C
:100D00000034FF3400340034FF34FF34FF34FF3448
:100D10000034FF34003400340034FF340034003435
:100D2000FF34FF34FF34FF34FF34FF34FF34FF342B
:100D3000FF34FF34FF34FF34FF34FF34FF34FF341B
:100D40000034FF3400340034FF34FF34FF34FF3408
:100D50000134FF34013401340034FF3400340034F2
:100D60000034FF3400340034FF34FF34FF34FF34E8
:100D70000134FF34013401340034FF3400340034D2
:100D80000034FF3400340034FF34FF34FF34FF34C8
:100D90000034FF34003400340034FF3400340034B5
:100DA000FF34FF34FF34FF34FF34FF34FF34FF34AB
:100DB000FF34FF34FF34FF34FF34FF34FF34FF349B
:100DC0000034FF3400340034FF34FF34FF34FF3488
:100DD0000134FF34013401340034FF340034003472
:100DE0000034FF3400340034FF34FF34FF34FF3468
:100DF0000134FF34013401340034FF340034003452
:100F00000D347734773477342E346434693467346D
:100F10006934743461346C342D346234613468342F
:100F20006E342E34643465340D3453346E346F347F
:100F30006F34703479342034563430342E343634AF
:100F40003434203444344334433420342034203483
:100F500020342034203420342034203420342034F1
:100F600020342034203420342034203420340D34F4
:100F7000303438342E3432343034303438340D3464
:084000000200000006000400AC
:02400E00543D1F
:00000001FF
